:1000000061288F00220884002009282084138F088B
:1000100003195C28F03091000E0880389000F03011
:1000200091030319910003198F0303195C28182801
:100030002B2003010C1820088E1F20088E0803199E
:100040000301900F252880060C28262800000F2881
:10005000841780055C280D080C0403198C0A803075
:100060000C1A8D060C198D068C188D060D0D8C0D35
:100070008D0D5C288F018E00FF308E07031C8F07CB
:10008000031C5C2803308D00DF3048203C288D01A4
:10009000E83E8C008D09FC30031C51288C070318A6
:1000A0004E288C0764008D0F4E280C1857288C1C86
:1000B0005B2800005B28080083130313831264008D
:1000C00008008316FF3085000C308600831206136B
:1000D000831606138312861283168612831201304A
:1000E000A600640006302602031896280630A200F7
:1000F0001030A00050308E000430012064308E009B
:100100000230012086108316861083120610831693
:100110000610323083123A2086148316861083121A
:100120000614831606108312A60F71280630A2004B
:100130001030A00064308E000430012078308E0032
:100140000230012050308E00023001205A308E00E3
:100150000230012086108316861083120610831643
:10016000061083126400051EBA28061483160610B2
:100170008312BE2806108316061083126400851DA4
:10018000C6288614831686108312CA288610831602
:0A01900086108312B2286300CB280A
:02400E00F53F7C
:00000001FF
